:040000002500540A79
:100020006100B6021602E2010000170A1F0A000072
:100030000000000000000000340A0000340A7600CE
:10004000210A220A340AC106100A0000000000003A
:1000500000000000000000000000000000000000A0
:10006000000000000000000072000C02E201C90A5A
:10007000DC0AE70AF20AFD0AF20AFD0AF20AFD0AA0
:10008000F20AFD0AF20AFD0AF20AFD0AF20AFD0A64
:10009000F20A0B0B190B240B2F0B3A0B450B500BD1
:1000A000600B6B0B7A0B850BFC0C0600000C26001A
:1000B000070C2400110C2B0075006C006A006D0009
:1000C0006E006F007000710076006909C50C0200B7
:1000D000A00A840C3700F80C3800F90C3900FA0C2F
:0800E0003A00FB0C3B00000894
:1001400023096607AE0AF207B20207040304FC0C97
:10015000D2010307070500000000A10A2309660673
:10016000A00AF207B20207040304FC0CD201030741
:10017000070500000000AF0A110C2B006C006A009C
:100180006D006E006F00700071007200F00C67016E
:1001900000080000000000000707D70AEB02D40A9D
:1001A000110C2B00AC020008000000000008110C2C
:1001B0002B00000000000008F502DF0A540A0000CE
:1001C0000000000000000706E60AAC02000800007C
:1001D0000000000000000000000000000706BC0A4C
:1001E000AC020008AC02030407060305710300001B
:1001F00000000000000000000008000000000000F7
:100200000000AC020707080B1107BC0A0000000839
:100210001106BC0A0008AA020A02EC010000000054
:100220000707160B1107BC0A000000081106BC0ADC
:1002300000080706BC0AAC02AA0200000000000089
:1002400000000000000000080706BC0A11022D0093
:10025000030C2C000000000000000000000807064E
:10026000BC0AAC02AA02000000000000000000006E
:10027000000000080706BC0A11022E00030C2C0027
:1002800000000000000000000008AC02AA0200000C
:100290000000000000000000000000000000000856
:1002A00011022F0007065B0B030C2C00000000005E
:1002B0000000000000086C006A0070007100990BDB
:1002C000AC02AA02000000000000000000000000D4
:1002D000000000000008110230000706760B030C36
:1002E0002C00000000000000000000086C006A0004
:1002F0007100990B0707BC0AAC02AA0200000000BB
:10030000000000000000000000080707BC0A6C00A5
:100310006A002704C7040D0243068F0B5D0AC70558
:10032000910B73006D006E006F00700071006A0029
:10033000A00AFF0F0D028E018F019001910143076A
:10034000910B750017028D014306A70B910B180244
:100350008E014307B00BFC0C0600000C2600910B2D
:1003600019028E014307B90BFB0C0600000C260096
:10037000910B1A028E014307C20BEB0C0600000C16
:100380002600910B1B028E014307910BDE0C060029
:06039000000C2600910B99
:0407F800A304540AF8
:021FFE00EA0FE8
:00000001FF
